:100000004F28A00046202730A200103032202008C0
:10001000800484138006A201A101841720088006B1
:10002000000080068413000503191C282508A10779
:100030000318A20F0D28A20322084B288001840A6E
:10004000FF3E031D1E284B28A401A300FF30A30779
:10005000031CA407031C4B280330A200DF3032200E
:100060002628A201E83EA100A209FC30031C3B287F
:10007000A10703183828A1070000A20F382821186B
:100080004128A11C45280000452808008004482874
:10009000FF3A841780058313831203130800073087
:1000A00099002030840040301E2030308500CB3055
:1000B000831685000230960095008113013083126B
:1000C000A400F4302520051585120130A400F43079
:1000D0002520851605120130A400F43025208B134D
:1000E0008B1505158516051683108518831483183E
:1000F0002C14831C2C100508AB000B1063000A3075
:10010000242003018518013E2C18013C031D892879
:100110007128851232302420A7013C30A600051535
:10012000851605160A3024208C30A5000530840081
:1001300001300120AA00A1302A02031CA6280511C3
:100140000A30242085120A3024200512A901143017
:10015000A8000130AB00FB302B020318C5280301B7
:100160008518013E2C18013C0319C02883108518FE
:10017000831483182C14831C2C10A7013C30A60078
:1001800004302420AB0A031DAB28A603260A03195A
:10019000A70327082604031DCE287128A803280AD0
:1001A0000319A90329082804031DA9288F28D72883
:02400E00A43FCD
:00000001FF
